:020000023000CC
:10E000000D9472F00D949BF00D949BF00D949BF089
:10E010000D949BF00D949BF00D949BF00D949BF050
:10E020000D949BF00D949BF00D949BF00D949BF040
:10E030000D949BF00D949BF00D949BF00D949BF030
:10E040000D949BF00D949BF00D949BF00D949BF020
:10E050000D949BF00D949BF00D949BF00D949BF010
:10E060000D949BF00D949BF00D949BF00D949BF000
:10E070000D949BF00D949BF00D949BF00D949BF0F0
:10E080000D949BF00D949BF00D949BF00D949BF0E0
:10E090000D949BF00D949BF00D949BF00D949BF0D0
:10E0A0000D949BF00D949BF00D949BF00D949BF0C0
:10E0B0000D949BF00D949BF00D949BF00D949BF0B0
:10E0C0000D949BF00D949BF00D949BF00D949BF0A0
:10E0D0000D949BF00D949BF00D949BF00D949BF090
:10E0E0000D949BF011241FBECFEFD1E2DEBFCDBF58
:10E0F00001E00CBF12E0A0E0B2E0E2E7F1EF03E0E4
:10E100000BBF02C007900D92AC36B107D9F722E0E1
:10E11000ACE6B2E001C01D92AC37B207E1F70F9454
:10E120000FF20D94B7F801E20EBF0FEE0DBF1124F0
:10E130001FBE0D940FF20D9400F020917A023091E1
:10E140007B022115310561F48093C6008091C000E7
:10E1500086FFFCCF8091C00080648093C00008954A
:10E160002230310559F48093D6008091D00086FF8B
:10E17000FCCF8091D00080648093D00008959C01F2
:10E1800090E080E08217930709F40895EFECF7E040
:10E190003197F1F700C000000196F4CFE0ECF0E019
:10E1A00080818260808320E12093C40098E1909375
:10E1B000C100E0EDF0E08081826080832093D40094
:10E1C0009093D1000895019719F480E885B90895D6
:10E1D00015B8089581B1806F81B982B1806F82B91D
:10E1E0006D9A75989D9AA598E1E0F1E0808188622A
:10E1F0008083E2E0F1E080818862808308958F98D7
:10E2000008958F9A0895CF93DF93C82FD62F662352
:10E2100009F448C05D9AC7FF47C0A39A80910201E4
:10E22000C6FF44C0806880930201C5FF41C0A49A24
:10E23000C4FF40C08D9A00C00F9401F182E08A951E
:10E24000F1F700C00F94FFF0C3FF36C0A39A80918E
:10E250000201C2FF33C0806880930201C1FF30C059
:10E26000A49AC0FF2FC08D9A00C00F9401F192E0D4
:10E270009A95F1F700C00F94FFF0A39A80910201E4
:10E28000806880930201A49A8D9AD1111DC0C43078
:10E29000D8F48FE999E10197F1F700C00000DF9110
:10E2A000CF9108955D98B7CFA398B8CF8F77BBCFA4
:10E2B000A498BECF8D98BFCFA398C9CF8F77CCCF6E
:10E2C000A498CFCF8D98D0CF95ED9A95F1F7E6CF62
:10E2D00060E00D9403F180580D9468F181E00D9495
:10E2E00068F182E00D9468F161E00D9403F1CF9341
:10E2F000DF93EC018991811103C0DF91CF910895E3
:10E300000F9474F1CE01F5CFCF93DF93EC01FE01B2
:10E3100084912196811103C0DF91CF9108950F94CC
:10E3200074F1F5CF879A559A9B9AE1E0F1E08081EC
:10E33000806880839C9A859A0F94FFF05D98A39AD9
:10E34000E2E0F1E0808180688083A49A8D9A8FE575
:10E350009AEE0197F1F700C00000A39880818F77B3
:10E36000808300C00F9401F192E09A95F1F700C00C
:10E370000F94FFF08FE090E40197F1F700C00000E8
:10E380000F9401F192E09A95F1F700C00F94FFF01D
:10E390008FE891E00197F1F700C000000F9401F1C0
:10E3A00092E09A95F1F700C00F94FFF085ED8A9501
:10E3B000F1F700008D9800C00F9401F192E09A955A
:10E3C000F1F700C00F94FFF085ED8A95F1F700009A
:10E3D0008D9800C00F9401F192E09A95F1F700C07A
:10E3E0000F94FFF082E08A95F1F700C0A39A00C075
:10E3F0000F9401F192E09A95F1F700C00F94FFF0AD
:10E4000085ED8A95F1F7000088E00F9468F10F948C
:10E410006EF186E00F9468F18CE00D9468F1CDB751
:10E42000DEB7CA53D1400FB6F894DEBF0FBECDBFE2
:10E4300094B7F894A89514BE809160008861809389
:10E44000600010926000789493FFA9C08091FC1F37
:10E450009091FD1FA091FE1FB091FF1F8A3A954534
:10E46000AA4AB545A9F44091F41F5091F51F609157
:10E47000F61F7091F71F6A017B01E3E03E2E31E049
:10E4800015E001E18091F81F9091F91F009771F458
:10E4900000008091C0008D7F8093C00081E1809357
:10E4A0005700E895EE27FF270994FFCF2091FB1F27
:10E4B00020FF09C0F601E0925B0030925700E8951A
:10E4C00007B600FCFDCF46015701AFEF9A1AAA0A22
:10E4D000BA0A21FF52C024708091F81F9091F91F51
:10E4E000009729F0481559056A057B0578F0F60173
:10E4F000E0925B0010935700E89507B600FCFDCF53
:10E5000000935700E89575016401BCCF4090F01F5F
:10E510005090F11F6090F21F7090F31F222331F191
:10E520006BBEF201A791B6910D01FA0160935B00F9
:10E5300030935700E89511244E5F5F4F6F4F7F4F28
:10E54000B2E04B0E511C611C711C8330910590F0A0
:10E5500002974092F01F5092F11F6092F21F70924A
:10E56000F31F9093F91F8093F81FB6CFF201A0819B
:10E57000B181DACF80E090E0ECCF5F5F6F4F7F4FEB
:10E580008130E1E09E0730F09A959093F91F8093D7
:10E59000F81FB9CF1092F91F1092F81FB4CF109244
:10E5A0007B0210927A02279A2F9A8091C000826093
:10E5B0008093C00080E18093C40088E18093C10013
:10E5C00000000F94EAF080E885B90F94CEF00F9424
:10E5D00092F10F946EF180E00F946BF181E40F944F
:10E5E0006BF183E092E00F9477F187E10F946BF188
:10E5F00086E192E00F9477F185E60F946BF185E266
:10E6000092E00F9477F115B810E000E0C12CD12C06
:10E61000760137EC832E3BE1932EA12CB12C809117
:10E62000C00087FD07C08091D00087FD03C00115A1
:10E630001105A1F08091D00087FF06C082E090E034
:10E6400090937B0280937A02012B09F49CC4279853
:10E650002F9884E690E00F94BFF01ACFF5E0FA957A
:10E66000F1F700002FEFC21AD20AE20AF20A81E0A3
:10E6700031E2C3163EE4D306E104F10408F480E07D
:10E68000082F10E0C701B601A50194010F9452F8BC
:10E69000C65DDE4F688379838A839B83CA52D140EB
:10E6A000672B682B692B09F0BACF85B1805885B9E3
:10E6B000B6CF60917A0270917B02CC24C39422E1A0
:10E6C000D22E2AE7E22EF12C61157105A9F42091D2
:10E6D000C00027FD2DC0B1E0CB1AD108E108F10838
:10E6E00099F7EBBEF601C790D690CD20C09429F3E0
:10E6F000EE27FF270994DDCF6230710561F7209185
:10E70000D00027FFE8CF6091D600A33009F44CC1B8
:10E7100090F4A13009F439C1A23009F43EC1AA2312
:10E7200009F42DC120E030E02130310509F0C1CFDE
:10E730006091C600EACFA53009F449C1A63009F4BA
:10E7400064C1A43009F434C1A73061F7452B81F4CA
:10E750000F946EF184E10F946BF189E292E00F94D3
:10E7600077F18DE20F946BF18DE392E00F9477F1E6
:10E770008091760290917702A0917802B09179020F
:10E78000892B8A2B8B2B09F049C0CF5CDE4F288167
:10E790003981C153D1402F5F3F4FCF5CDE4F39836A
:10E7A0002883C153D1402B303105C0F1C25DDE4F0B
:10E7B00088819981CE52D1400196C25DDE4F998306
:10E7C0008883CE52D140069730F0C25DDE4F198269
:10E7D0001882CE52D1408BE50F946BF181E592E027
:10E7E0000F9477F1C25DDE4FA881B981CE52D1403E
:10E7F0008A2F845A149738F082E6C25DDE4FB881C2
:10E80000CE52D1408B1B0F946BF18AE20F9474F1BE
:10E81000CF5CDE4F19821882C153D14080917602BD
:10E8200090917702A0917802B0917902892B8A2B7E
:10E830008B2B09F48DC080916C0290916D02009732
:10E8400009F486C0019739F488E50F946BF188E5E7
:10E8500092E00F9477F180916C0290916D02029793
:10E8600039F487E50F946BF18FE592E00F9477F11F
:10E87000209172023091730240917402509175029E
:10E88000A4E6B0E00F947BF8CA5DDE4F688379831D
:10E890008A839B83C652D1402091760230917702C1
:10E8A00040917802509179020F9452F8C901CB5CE3
:10E8B000DE4FE881C553D140C25EDE4FE883CE51C2
:10E8C000D140CA5CDE4FF881C653D140C15EDE4FF5
:10E8D000F883CF51D140C95CDE4F2881C753D14066
:10E8E000C05EDE4F2883C052D140C85CDE4F388105
:10E8F000C853D140CF5DDE4F3883C152D140EEE1E5
:10E90000F1E0EC0FFD1F339620E2181619063CF4D7
:10E910006AE070E00F943EF820E3280FCB012293C9
:10E92000CE5DDE4FA881B981C252D140AE17BF077C
:10E9300059F7C75CDE4F8881C953D140C65CDE4FB2
:10E940009881CA53D1400F9477F185E20F9474F106
:10E950002981243109F480C008F06EC0263009F402
:10E96000BFC108F057C0223009F487C1233009F431
:10E9700074C1213009F459C180EC8A83C8C16B315C
:10E9800009F0D0CE1BE1A1E0CDCE1627C05DDE4F51
:10E990006883C053D140A2E0C5CE862F90E0982F67
:10E9A00088271627A3E0BECE862B1627A4E0BACE72
:10E9B0006E3071F51627C65DDE4F1882CA52D140FF
:10E9C000C55DDE4F1882CB52D140A5E0ABCEC65D0F
:10E9D000DE4F28813981CA52D1402F5F3F4FC65D3B
:10E9E000DE4FE881F981CA52D140E20DF31D608308
:10E9F00016272817390709F03AC3C65DDE4F9983F9
:10EA00008883CA52D140A6E08DCE611709F49ECE0C
:10EA1000A0E088CE223109F459C1233109F485C11F
:10EA2000203109F42AC101E0213109F0A5CF1A8271
:10EA300082E0E82EF12C9DC02A3109F424C108F0AF
:10EA400070C0283109F42DC108F057C0253109F4F0
:10EA50006CC1263109F090CF8A819B819827892744
:10EA600098277C01F3E0EF0EF11C1A82243109F0A3
:10EA70004DC2409176025091770260917802709178
:10EA80007902452B462B472BF9F08C0130E020E032
:10EA9000411451046104710409F023C240916C02D5
:10EAA00050916D024130510509F01BC242E050E027
:10EAB00050936D0240936C020093720210937302A4
:10EAC0002093740230937502D1016BBEF20127913D
:10EAD000369112962C931297FD01349613963C931F
:10EAE000139722E0420E511C611C711C0297129672
:10EAF000009759F7108200E03CC0293109F03CCF63
:10EB00008D81836C99E0E1E0F0E0082E909357004E
:10EB1000E89587B7082F017080FDFBCF1A821B8212
:10EB2000A8C02D3181F0213709F4F3C02B3109F051
:10EB300023CF8D81882309F4A2C0813009F4A1C0BC
:10EB400081E01A82A7C09D81903309F056C08F8161
:10EB5000882309F466C0813009F465C081E01A8217
:10EB60001B829C831D828E831F8200E0B7E0EB2E08
:10EB7000F12C8BE10F949DF0C05DDE4F8881C05376
:10EB8000D1400F949DF08F2D0F949DF0C05DDE4F0E
:10EB90001881C053D1401F258E2D0F949DF01E2546
:10EBA0008EE00F949DF085E11827E20CF31CCD5CFC
:10EBB000DE4FC880C353D140CC5CDE4FD880C453F5
:10EBC000D140EC14FD0409F0CCC1812F0F949DF0CD
:10EBD000C05DDE4F2881C053D1402F5FC05DDE4F46
:10EBE0002883C053D14085B1805885B941E050E0B9
:10EBF00001112DCD30E020E036C2892F807509F457
:10EC0000AECF89E0F0E0E0E0903539F080E0983573
:10EC100009F0A5CF89E0E3E0F0E08093570084910C
:10EC20009ECF8EE19CCF88E99ACF1A8288E08B83B1
:10EC300081E48C8386E58D8382E58E8389E48F83EE
:10EC400083E5888780E589878FE58A8782E38B87DC
:10EC500000E0ABE0EA2EF12C8CCFEA81E05980E0B5
:10EC6000E33020F4F0E0E050FE4F80811A828B8385
:10EC700000E0E3E0EE2EF12C7CCF00E0D8CE8EE178
:10EC800060CF88E95ECF1A8289E0E1E0F0E080930E
:10EC9000570084918B831C8200E0F4E0EF2EF12C6E
:10ECA00068CF8B81803571F48C81883039F489E0AC
:10ECB000E2E0F0E080935700849143CF89E0F0E0F8
:10ECC000E0E0F8CF89E0E3E0F0E0F4CF80EC8A8385
:10ECD00000E072E0E72EF12C812C912C540149CFF9
:10ECE0008A819B81AC81BD81BC01CD010F9474F8F8
:10ECF000CA5DDE4F688379838A839B83C652D14085
:10ED00002B013C01440C551C661C771C1A8200E048
:10ED10008FCE8A81809376028B81809377028C815B
:10ED20008093780210927902F1CF0A811B8110271B
:10ED300001271027233109F09BC080917602909122
:10ED40007702A0917802B0917902892B8A2B8B2BC4
:10ED5000F9F0411451046104710409F055C0C8016F
:10ED6000B0E0A0E08093720290937302A0937402CB
:10ED7000B093750281E090E090936D0280936C02F5
:10ED800040926E0250926F02609270027092710215
:10ED9000811490EE990693E0A906B10470F483E023
:10EDA000F401A0925B0080935700E89507B600FC41
:10EDB000FDCFAFEF9A1AAA0ABA0A4114B0EE5B0669
:10EDC000B3E06B06710408F0A1CF8B85DE011196CC
:10EDD000B301A20121E01B969C911B970C01FA0143
:10EDE00060935B0020935700E89511244E5F5F4FBE
:10EDF0006F4F7F4F0250110912960115110539F11D
:10EE00001A968C911A97E7CF80916E0290916F02BB
:10EE1000A0917002B091710284159505A605B70501
:10EE200009F4AECF8091720290917302A0917402A6
:10EE3000B0917502800F911FA11DB11D80937202C8
:10EE400090937302A0937402B093750299CF85E0FA
:10EE5000F20160925B0080935700E89507B600FCD2
:10EE6000FDCF81E180935700E8952A013B014ECF09
:10EE7000D301C201B695A795979587956C01F801C6
:10EE8000E80FF91FCA5DDE4FF983E883C652D1400F
:10EE9000CC5DDE4F8881C452D140CB5DDE4F98817E
:10EEA000C552D140CA5DDE4FE881F981C652D140DA
:10EEB000EC15FD0559F430E020E0000F111F221F72
:10EEC000331F400E511E621E731E20CFDC016D9158
:10EED0007D01C6010F94A9F8BFEFCB1ADB0AC70169
:10EEE000E1CF40917202509173026091740270916F
:10EEF0007502400F511F621F731F4093720250939F
:10EF000073026093740270937502DECDF1016101AA
:10EF1000C80ED91EB301A20141BD052F162F272F00
:10EF2000332702BD4F5F5F4F6F4F7F4FF89AA0B5F9
:10EF3000A2833196CE16DF0679F7AC014150510914
:10EF400070E060E04F5F5F4F6F4F7F4F440E551E84
:10EF5000661E771EE3E0F0E0EC0FFD1FE80FF91FDF
:10EF6000C9CDD601ED916D01CA5DDE4FE883C65271
:10EF7000D1408E2F0F949DF0CA5DDE4FF881C652AE
:10EF8000D1401F271ECEC25DDE4F19821882CE529D
:10EF9000D140CF5CDE4F19821882C153D140C05D91
:10EFA000DE4F1882C053D14010E0C65DDE4F19829B
:10EFB0001882CA52D14050E040E0812C912C54017B
:10EFC000412C512C320121E030E0CE0101961C0190
:10EFD000CD5CDE4F8883C353D140CC5CDE4F38829A
:10EFE000C453D140DE01A25EBE4FCE5DDE4FB98379
:10EFF000A883C252D140B0916702CB5CDE4FB88388
:10F00000C553D140E0916802CA5CDE4FE883C65325
:10F01000D140F0916902C95CDE4FF883C753D140FB
:10F0200080916A02C85CDE4F8883C853D140CE5DB0
:10F03000DE4F9881C252D140C75CDE4F9883C953DE
:10F04000D140CD5DDE4FA881C352D140C65CDE4FBA
:10F05000A883CA53D140FE013B96CC5DDE4FF983B5
:10F06000E883C452D14090E080E0A0E05DCBC65D73
:10F07000DE4F39832883CA52D14054CB97FB072EE9
:10F0800016F4009407D077FD09D00F9486F807FC9A
:10F0900005D03EF4909581959F4F089570956195A8
:10F0A0007F4F0895A1E21A2EAA1BBB1BFD010DC0C4
:10F0B000AA1FBB1FEE1FFF1FA217B307E407F50728
:10F0C00020F0A21BB30BE40BF50B661F771F881F04
:10F0D000991F1A9469F760957095809590959B019A
:10F0E000AC01BD01CF0108956927962769277827CC
:10F0F0008727782708950F949AF8A59F900DB49FBD
:10F10000900DA49F800D911D11240895AA1BBB1B77
:10F1100051E107C0AA1FBB1FA617B70710F0A61B17
:10F12000B70B881F991F5A95A9F780959095BC0138
:10F13000CD010895A29FB001B39FC001A39F700DA0
:10F14000811D1124911DB29F700D811D1124911DEF
:10F150000895262FF999FECF1FBA92BD81BD20BD1B
:10F160000FB6F894FA9AF99A0FBE01960895F8949A
:02F17000FFCFCF
:10F172000F020A4F726967696E616C204265727391
:10F1820065726B6572004D696D69722052657365B7
:10F1920061726368002E2E2E0020446F206E6F7401
:10F1A20020646973636F6E6E65637421002055700D
:10F1B20067726164696E67206669726D77617265F4
:10F1C200007C202020207C00777269746520007604
:0CF1D20065726966792000202020000092
:040000033000E000E9
:00000001FF
